:10000000020108E5F06011ECA2E713FCED13FDEE30
:1000100013FEEF13FFD5F0EF22C236120B98120F2A
:100020005C220002002EFF562B16000209C8C0E019
:10003000C0D075D008309906C299D231801C309852
:1000400019C29885992FD230E52FB4330DC2ADC2B5
:10005000CAD232C2BDD2BC439104D0D0D0E0328DDE
:100060007DC2A61216D6AF7D1216D6D2A622FF02E8
:1000700016D600C0E0C0F0C083C082C0D075D010DA
:1000800053917FAA300530BA7801D350030200FDA6
:10009000E4F5305391FBE534B40006E535B4FF01D7
:1000A000D35008203505757C46800FE534B4010A2D
:1000B000E535B40005757C45C235AF7C12186D126C
:1000C0001954C220C221C223C222C251C2531219E2
:1000D00016C228C229C22BC22AC252C254121908FF
:1000E0001216A2121814D2621216FAC23FC2451298
:1000F0000C68120407C2BCD2BDD2CAD2ADD0D0D0D7
:1001000082D083D0F0D0E0327581D5E4787FF6D804
:10011000FD900F4AE4937002804EC31392D5C3132F
:1001200092D1FFA3E493F8B0D5402130D505E4A3E4
:1001300093F5A0E420D102A39320D507F608DFF3BE
:10014000A380D1F208B800F605A080F2E80303030B
:10015000541F2420F9E85407F8E4D333B800028090
:100160000333D8FD47F780D875A0FF53F1F343A4BC
:100170001075D4CF5380F375D57F43A5C075A6F60F
:10018000D2A375A7F275E10375E24075B1677558A2
:100190000BE5B160FC75A90175EF0675D900758E88
:1001A00009758A00758BEA758C00758DEA75892151
:1001B00075884075C80075CAB475CBFF75CCB47529
:1001C000CDFF75910075920075930075940075953B
:1001D0000043E680759810758700D2AFD2AC75A148
:1001E0004075A20075F801752D1AE4F52EC299D25A
:1001F000BDD2A512169A121908120C681216A21274
:100200001586121180D2ADD2CAD2A71204071218D5
:1002100014754B011216FAC223C22230A303303BDD
:100220000BC23B852D83852E821202717981770066
:100230007981B70401D350E320300330320479814F
:1002400077007981E7600E14601014601214601456
:1002500014601680171205C78012120DA0800D12AF
:100260000E99800812001980031216FA798107800E
:10027000BFC082C08322E58124FEF9EFF887F0A495
:10028000FFE7C5F0CEFAA42EFE500205F0E7C5F058
:10029000CDFBA42DFD500205F0E7C5F0CCA42CFC4D
:1002A00019E7601688F0A42EFEE5F03DFD50010C24
:1002B00087F0EA121966EBA42CFC19E7600988F0B4
:1002C000121966EAA42CFC19E7600588F0A42CFC3E
:1002D0000203A21203F8C380021819E637F6DAF90E
:1002E00092D50203A2BC000EBE0032EF8DF0842036
:1002F000D226FFADF0227B0075F008EF2FFFEE3322
:10030000FEEB33FBEE9DEB9C4005FBEE9DFE0FD517
:10031000F0E9E4CECDCBCC227EFF7FFF22EDB410FE
:10032000005022EE8DF084FEEF54F045F0C48DF0C5
:1003300084C4FCEF540FC445F0C48DF084FFADF0CD
:10034000E4CC4FFF22EE8DF08420D2CC7E08CEC5C7
:10035000F0CDCBEF2FFFED33FD10D7079B5005D528
:10036000F0F1229BFD0FD5F0EA22C3E49FFFE49E4B
:10037000FE22C3E49DFDE49CFC22E58124FBF9E51B
:10038000D054184404F87A04E687F0B5F00A090856
:10039000DAF6E4FEFF0203A2E45004FE0480F5F462
:1003A00080F174FCD083D0822581F581C082C08326
:1003B00022E4FEFFEB700122239003BB73800880D0
:1003C0000F801A8002801FE70912197970F98022C4
:1003D00089828A83E0A312197970F98015E30912E2
:1003E000197970F9800C89828A83E493A3121979B0
:1003F00070F81FBFFF011E22E5D054182407F8E54E
:100400008124FCF97A0422E540B54206E541B54372
:1004100001D34015E541C39543F560E5409542F5AC
:100420005F8542618543628013E543C39541F56072
:10043000E5429540F55F854061854162AE5FAF6002
:10044000E4FCAD441202E58E638F64756500E565DA
:10045000B54400504EE5652401FFE433FEAC63ADC6
:1004600064EF8DF0A4CFC5F0CCA42CFCEE60038D1E
:10047000F0A42CFEEF2562FFEE3561C0E0EFC0E096
:10048000E5652565240012194CA3D0E0F092D6153D
:1004900082C582B4FF021583C582A2D6D0E0F005E2
:1004A0006580AB2290000012189C4005E4F55B804B
:1004B00037755C00E55CB54400502D255C240012C6
:1004C000194C8EF0E0B5F0078FF0A3E0B5F00050C6
:1004D00013E55C25E0240212194C12189C4005E536
:1004E0005C04F55B055C80CCE54425E024FEF582E8
:1004F000E434FFF58312189C5006E54424FFF55BB5
:1005000079CA78CBE7F679C978CAE7F679C878C9A5
:10051000E7F679C778C8E7F6A75B86F0E7B5F02578
:1005200079C987F078C7E6B5F01B78CA86F078C736
:10053000E6B5F01178CB86F078C7E6B5F00779C05C
:10054000A75BAF5B2279C0E7FF224E6575686175D6
:100550007320456C656374726F6E69637300536FCB
:10056000756E64204D6F64756C2C56657273696F7F
:100570006E20332E322E32303130205243006D65E2
:100580006D6F72792073697A653A20756E6B6E6F44
:10059000776E006D656D6F72792073697A653A20A8
:1005A000344D42006D656D6F72792073697A653ADA
:1005B00020384D42006D656D6F72792073697A65E0
:1005C0003A2031364D42002030030209C7C230E5DF
:1005D0004C64016006203403020730E54CB401028C
:1005E000800302071F30340302071FC2CAE4F5303C
:1005F000E535121988E5343400F583E52FF005352B
:10060000E53570020534C235E534B40102800302D9
:10061000071FE535B40002800302071FC036C0374C
:10062000C038C039E433E4500114C0E0C0E0E4C095
:10063000E0C033FC7D01FEFF12027612037ABF0098
:1006400033C2967F061218B11216E3C2967FD812F3
:1006500016D675F0101218D51200031216D675F0C2
:10066000081218D51200031216D6AF391218B1129B
:1006700016E30533C2967F061218B11216E3C2962E
:100680007F021216D675F0101218D512000312163A
:10069000D675F0081218D51200031216D6AF39120B
:1006A00016D6E4F55FF56012190E3400F583E012FA
:1006B000006E0560E560B400EED2961216E3C03617
:1006C000C037C038C039E4FCFD7E01FF1202D38C74
:1006D000368D378E388F39C036C037C038C039E4D0
:1006E000FC7D3F74FFFEFF12037ABFFF0280247F70
:1006F0004512186D5391FBF595F594C2BCD2BD120D
:1007000019081216A2120C68120407E4F54A43EF06
:1007100010800C7F40120C5EE4F534F535D2353094
:10072000340DE54C7009D2CAAF2F120B0CC2342223
:10073000E52FB437030207F0501AE52F24D07003D9
:100740000207CC24FC602414700302099114700386
:1007500002096522E52F24C8700302090324FE70F4
:100760000302099814700302099B22D231C2CAC243
:1007700096E4FFFDFB1216BBE4F559F55AF55BF55F
:100780005C20310280FBE412006E79C0A7A33030F8
:1007900007E52FB43902802F79C0E7FF120C5E0500
:1007A0005CE55C700E055BE55B7008055AE55A7008
:1007B000020559C059C05AC05BC05CE4FFFCFE7D15
:1007C0004012037ABF00BAD296D2CA22203211D286
:1007D000BDC2BCD2ADD2CA5391FB7F47120C5E2280
:1007E000754C01C232E4F534F535F5331219702237
:1007F00079C1B70100500974FFF55DF55E0780F01F
:100800001219967F0D120C5E7F0A120C5EC2CA127C
:1008100019967B057A05794A1203B11218B7C0E020
:10082000EFC0E078C1E6FFD0E0FDD0E01218245020
:100830000EE690054A93FF120C5E79C10780D37FC4
:100840000D120C5E7F0A120C5E1219967B057A055A
:10085000795E1203B11218B7C0E0EFC0E078C1E6CC
:10086000FFD0E0FDD0E0121824500EE690055E9314
:10087000FF120C5E79C10780D37F0D120C5E7F0AD8
:10088000120C5EC2967F9F1216D6E412006EE4121E
:10089000006EE412006EE5A324EA600280301219B3
:1008A000967B057A0579931203B11218B7C0E0EF71
:1008B000C0E078C1E6FFD0E0FDD0E0121824503E41
:1008C000E690059393FF120C5E79C10780D312194D
:1008D000967B057A05797E1203B11218B7C0E0EF56
:1008E000C0E078C1E6FFD0E0FDD0E0121824500E41
:1008F000E690057E93FF120C5E79C10780D3D296F5
:10090000D2CA22C2CA79C1B72000500974FFF55D6E
:10091000F55E0780F012199690017CE079C2F7E746
:10092000FF120C5E79C3770079C287F078C3E6B511
:10093000F001D3502D79C4770079C4E7FE75F00932
:1009400079C3E7A42EFFE435F0FEEF247DF582EEB7
:10095000121960FF120C5E79C407B709DC78C30670
:1009600080C6D2CA22C2CAC205C215C2967F06126A
:1009700018B11216E3C2967FC71218B11216E37FA0
:100980000A120C5E7F0D120C5E7F2E120C5ED2CA14
:1009900022D2CAD234C23022D23B22C2CA12159508
:1009A0008E5D8F5EE55D455E70028014AF5D120C5A
:1009B0005EAF5E120C5E7F0A120C5E7F0D120C5E43
:1009C000E52FB43CD8D2CA22C0E0C0F0C083C082B8
:1009D000C0D075D018C2CF0557E557146012146007
:1009E00051147003020A74147003020ABA020B0154
:1009F000E52054406003020B017F227993E7FD124A
:100A0000005FE4A22292E0B40122D223C222304F3E
:100A1000153053081218E61217E0800D12129A12C0
:100A200012F1D225800912118A020B0112118A02D9
:100A30000B01E52254406003020B017F2179A5E7F9
:100A4000FD12005FE4A22A92E0B40122D22BC22A56
:100A50003050153054081219371217E0800D121457
:100A6000991214F0D22D8009121387020B01121370
:100A700087020B01E4A20192E0B401028003020BA1
:100A8000017F227993E7FD12005FE4A22292E0B495
:100A90000123D223C222304F173053081218E61216
:100AA00017E0800F12129A1212F1C24FD22580085D
:100AB00012118A804C12118A8047E4A21192E0B48C
:100AC00001377F2179A5E7FD12005FE4A22A92E0B9
:100AD000B40123D22BC22A305017305408121937D0
:100AE0001217E0800F1214991214F0C250D22D8008
:100AF000081213878003121387E4F557D24B754B06
:100B000001D0D0D082D083D0F0D0E0328F5F1218E5
:100B1000AA2485121894F5601218AA2484E5F034EA
:100B2000011218AA2483121894F561E561540F2468
:100B3000FFF5627401AB620B121923F563E5605493
:100B400020B42025E561540F601EE563554A700C02
:100B5000E563424AE56204FF1217B222E563F452EC
:100B60004AE56204FF1217E022E5605404F56412BE
:100B7000197F4023E564700DD248E561540FF53CC0
:100B8000D226855F4DE564B4040DD249E561540F6A
:100B9000F53ED22E855F5222E4FEFFA280925A30AB
:100BA0005964205A61C28C308D09C28D75730AD286
:100BB00058804EE573600BE57324FFF573E4FEFF88
:100BC000803FE58CFBEF2BFFE43EE58AFDE42DF949
:100BD000E43FFEE9FFBE2303B928004009BE5504E7
:100BE000BFF001D3400A757414E4FEFFD25880119F
:100BF000E574600BE57424FFF574E4FEFF8002C227
:100C0000581219438003E4FEFFA25A92598E598F5D
:100C10005AE559455A6046AE59AF5A1204A4E54602
:100C20002F24022545F549303D0CC23DD23FE4FF5B
:100C3000120B0CD24A22303E0AC23EC23F7F011242
:100C40000B0C22303F17E549B54805204A02800ABF
:100C5000120D44AF49120B0CC24A854948228F99A4
:100C600020310280FBC23122755F0012197F4031B2
:100C70001218AA248512189454886408701FD2454B
:100C8000855F461218AA2484121894543FF5441222
:100C900018AA248D121894543FF5458004055F80EE
:100CA000CA204503020D2A75F00990017CE0A424B6
:100CB000F7FEE5F034FF79C5F709EEF7E724801277
:100CC00018DE787EF609E724811218DE787FF609AF
:100CD000E724821218DE7880F67F05120D2B755FEF
:100CE00000E55FB545005042756000C296797EE729
:100CF000FF787FE6FD7880E6FB1216BBE4FF121852
:100D0000B175F005E55FA42560FFE435F0FEEF1254
:100D10001988EE3400F583E5A3F07F01120D2B0551
:100D200060E560B405C5055F80B722797EE72FF7DF
:100D30008FF0E7B5F000500B797F07E770057980F9
:100D4000E704F722755B00E55BB54500505175F08F
:100D500005E55BA412198812188CB54801D3503BE5
:100D60001218CE247DF58212188CB54800402C1242
:100D700018CE247EF58212188CB54901D3501C126E
:100D800018CE247FF58212188CB54900400D121838
:100D9000CE2480F58212188CF54922055B80A822AA
:100DA000E4A22692E0B401028003020E7DC226E591
:100DB0002454026003020E55E5245401700F854D42
:100DC0004ED220AF4D121202D222D24F22C24F1267
:100DD000130EE550600CB40204E5516005E551B412
:100DE0000247E55064046041E5215401701EE54E60
:100DF000B54D0B121954C220AF3D1217E022AF4D72
:100E0000121202D222854D4E12195B22854D4FD20D
:100E100021E54FB54E0A203F06C221D24FD25322C0
:100E2000AF4D12120212195B22E551B40410854D28
:100E30004EAF4D121202D222D22012195B22E5507F
:100E4000B40411E5516005E551B40208AF4D12122A
:100E50000212195B22C24F12130EE551B40410C2E4
:100E600021854D4ED220AF4D12120212195B228500
:100E70004D4FD221AF4D12120212195B22E4A22172
:100E800092E0B40113E4A22392E0B4010B854F4E2B
:100E9000C221D220D205C22322E4A22E92E0B401C4
:100EA000028003020F2EC22EE52554027068E5254C
:100EB0005401700F855253D228AF52121401D22A16
:100EC000D2502212150DE555600CB40204E55660AF
:100ED00005E556B4023FE5235401701FE553B552B2
:100EE0000B121916C228AF3F1217E022AF5212148C
:100EF00001D22A855253D250D25222855254D2293D
:100F0000E554B55307C229D250D25422AF5212141D
:100F100001D250D2522212150DE556B40401228599
:100F20005254D229AF52121401D250D25222E4A20A
:100F30002992E0B40113E4A22B92E0B4010B855492
:100F400053C229D228D215C22B2223BD0308402721
:100F50001008424E2004D3FF04D4FF00A281925D0A
:100F600020600E305D0B75F90075FA00D2DE020FBD
:100F7000EA306073205D7053D8BF30DF0CC2DF12DF
:100F8000191D756D0AD25F8061E56D600BE56D24FA
:100F9000FFF56D12191D8052E5FAFBE56C2BFBE4A1
:100FA000356BF56B8B6CAA6CE5F9FDE42DF56CE403
:100FB0003AF56BB42305E56CB42800400DE56BB43D
:100FC0005506E56CB4F001D3400A756E1412191D74
:100FD000D25F8016E56E600BE56E24FFF56E121988
:100FE0001D8007C25F800312191DA25D9260AE6B67
:100FF000AF6C8E718F72E5714572700302111EE540
:1010000071B43206E572B4C801D35005756F018022
:1010100014E571B44205E572B468004005756F02CD
:101020008003E4F56F79D1B7FE01D3500107E56F76
:10103000B40109E5706402700302111AE56FB4028D
:1010400008E570B4010302111AE56F600F14700314
:101050000210BE1470030210ED02111AE56FB57094
:101060003379D2E714600624FE6015804F121930E0
:10107000401F79D3E7FF12112279D312184D803C1B
:10108000121930400C79D4E7FF12113D79D41218AF
:101090004D02111A79D2E724FE600724FE60110286
:1010A000111A79D3E7FF12112279D312184D806AF1
:1010B00079D4E7FF12113D79D412184D805CE56FA9
:1010C000B5701D121930402378D2E66402601C7995
:1010D000D2770279D3E7FF12112279D17700803AD3
:1010E00079D2770179D1770079D307802DE56FB573
:1010F000701D121930402378D2E66404601C79D246
:10110000770479D4E7FF12113D79D17700800B790C
:10111000D2770379D1770079D407856F7022305E5A
:1011200000228F5930450DE559240925442545FFF6
:10113000120B0C22E5592408FF120B0C228F593098
:10114000451EE5593395E06480B48006E559B40046
:1011500001D3400CE5590425442545FF120B0C2210
:1011600030450AE5597006203F03D23D2230450A3A
:10117000E5597006303F03D23E22AF59120B0C22C4
:1011800075F90075FA0075D90222E4A20592E0B45F
:10119000016FE4A22592E0B40105121339C22512B1
:1011A00012F1E4A22492E0B40104D222C224E4A207
:1011B0002292E0B40104304F0122798587F07882D1
:1011C000E6B5F03A788686F07883E6B5F030788731
:1011D00086F07884E6B5F026E4A20392E0B4011329
:1011E000798B7882E7F6798C7883E7F6798D788445
:1011F000E7F62212192AAF3D1217E0C20A22121393
:1012000039228F59755A01121832799212198D505C
:101210007CFA232A9012187302123302123B021234
:101220004302124B02125302125B02128D02128D04
:101230000212637992788EE7F680527992788FE77E
:10124000F6804A79927890E7F6804279927888E73A
:10125000F6803A79927889E7F680327992788AE74F
:10126000F6802A7992E7FF1213697992E730E31A40
:10127000E720E711755103E720E605755102800864
:1012800075510480087551018003755100055AE5B8
:101290005AB40A02800302120722304F53C24F7918
:1012A0008E788BE7F67982E6F7798F788CE7F67996
:1012B00083E6F77990788DE7F67984E6F779887890
:1012C00085E7F679897886E7F6798A7887E7F6857B
:1012D0005150A2049203A2029201A2099208AF3CCB
:1012E0001217B2305107AF3D1217E0C251853C3D95
:1012F00022C2967982E7FF7983E7FD7884E6FB12C4
:1013000016BBE4FF1218B17993A7A3D2052275F09A
:1013100009E54DA41218587992F7E730E317E72052
:10132000E70F755103E720E6047551022275510459
:10133000227551012275510022798207E7700979DF
:101340008307E77003798407798587F07882E6B5AB
:10135000F016788686F07883E6B5F00C788786F00C
:101360007884E6B5F002D22422EF20E104C20480A2
:1013700002D204EF20E004C2028002D202EF20E495
:1013800003C20922D20922E4A21592E0B40171E459
:10139000A22D92E0B40105121538C22D1214F0E40A
:1013A000A22C92E0B40104D22AC22CE4A22A92E038
:1013B000B4010430500122799787F07894E6B5F0B3
:1013C0003C789886F07895E6B5F032789986F07892
:1013D00096E6B5F028E4A21392E0B40113799D7863
:1013E00094E7F6799E7895E7F6799F7896E7F62266
:1013F000C228121916AF3F1217E0C21A221215386E
:10140000228F59755A0112183279A412198D507C05
:10141000FA232A9014177302143202143A02144267
:1014200002144A02145202145A02148C02148C023E
:10143000146279A478A0E7F6805279A478A1E7F63F
:10144000804A79A478A2E7F6804279A4789AE7F6F0
:10145000803A79A4789BE7F6803279A4789CE7F605
:10146000802A79A4E7FF12156879A4E730E31AE728
:1014700020E711755603E720E605755602800875CA
:10148000560480087556018003755600055AE55AC2
:10149000B40A02800302140622305053C25079A0CD
:1014A000789DE7F67994E6F779A1789EE7F6799545
:1014B000E6F779A2789FE7F67996E6F7799A789732
:1014C000E7F6799B7898E7F6799C7899E7F6855660
:1014D00055A2149213A2129211A2199218AF3E12A1
:1014E00017B2305207AF3F1217E0C252853E3F227B
:1014F000C2967994E7FF7895E6FD7896E6FB12169A
:10150000BBE4FF1218B179A5A7A3D2152275F00983
:10151000E552A412185879A4F7E730E317E720E75B
:101520000F755603E720E60475560222755604220D
:101530007556012275560022799407E7700979954E
:1015400007E77003799607799787F07894E6B5F006
:1015500016789886F07895E6B5F00C789986F0784C
:1015600096E6B5F002D22C22EF20E104C2148002EC
:10157000D214EF20E004C2128002D212EF20E40362
:10158000C21922D21922438909438E0153E4F84338
:10159000F103D28C22A280925C305B47205C44C273
:1015A0008C308D0EC28DE4F575F576757728D2589E
:1015B0008036E577600DE57724FFF577E4F575F57E
:1015C00076801BE58CFBE5762BFBE43575F5758B9A
:1015D00076AA76E58AFDE42DF576E43AF5751219DA
:1015E000438005E4F575F576A25C925BAE75AF7647
:1015F00022C20AC21AC2057993777FC207C215793F
:10160000A5777FC21722E4F55F756001C296FFFDE2
:10161000FB1216BBE412006EE5A390017CF0D2969B
:10162000F56175620090017CE0B56201D350030260
:101630001699856261E4F56375641075F0191218E6
:10164000BFFEE43FB40004BEFF01D3401175F019A2
:101650001218BFE43FF5651218F0F56780071218FD
:10166000F0F565F567C296AF66AD65AB671216BB60
:10167000E412006E12190E3401F583E5A3F0056043
:10168000E5607002055FD2960564E564B4190280D6
:101690000302163B05620216252279C074FFF70982
:1016A000F72279A777FF79CC770079D0770043A428
:1016B000C053803F43A53F5390C0228F688D698BF4
:1016C0006A7F031216D6AF6A1216D6AF691216D603
:1016D000AF681216D6228FA3E5F820E70280F953EF
:1016E000F87F22C2967F051216D6E412006EAEA3D2
:1016F000EE5401640160F3D29622306244C26285E6
:101700007859755A00E5595401600EE5795401B4D1
:101710000007AF5A1217428012E5595401B4000B6A
:10172000E57954016005AF5A12177AE559C313F5EC
:1017300059E579C313F579055AE55AB408C7857890
:101740007922BF04028027500DEF60161460161432
:10175000601614601622EF24FB60161460161460E5
:101760001622D28622D28722D29022D29122D292DF
:1017700022D29322D29422D29522BF0402802750F3
:101780000DEF601614601614601614601622EF2414
:10179000FB601614601614601622C28622C28722CD
:1017A000C29022C29122C29222C29322C29422C229
:1017B00095227E01EF60287565001218FDB5F018BE
:1017C0008BF0E565B5F01112187F04F0AB650BEEF8
:1017D000121923FE4278D2620565E565B408DB2262
:1017E0007E01EF602E7565001218FDB5F01E8BF0BE
:1017F000E565B5F01712187F14F012187F700DAB65
:10180000650BEE121923F4FE5278D2620565E56588
:10181000B408D5227A089003BDE4F0A3DAFCE4F51D
:1018200078F54A22F5F0E4B5F0078DF0EFB5F00158
:10183000D32275F009E559A4255AFFE435F0F55B8C
:101840008F5CE55C121988E55B1219602277FF79DD
:10185000D1770079D27700222409FBE435F0F559DD
:101860008B5AE55A121988E55912196022120C5E3A
:10187000E4F534F535F533C232F54C12197022E532
:101880006524BDF582E43403F583E022E5F03400FD
:10189000F583E022F582E5F012196022E08EF0B5C2
:1018A000F007A3E08FF0B5F00022E55F75F009A422
:1018B000221216D6D29622EF24FFFFEE34FF22E545
:1018C00062A42564FEE5F03563FFEE240122E55BAA
:1018D00075F005A422AC36AD37AE38AF3922F582AB
:1018E00019E712196022C24FC25312192AAF3C22C3
:1018F000E56275F019A4256404F566E422EF24FF7F
:10190000FBE434FFF5F0E4221215F1021606E5605F
:10191000121988E55F2279A5777FC21522E4F56B5D
:10192000F56C228002C333DBFC22C2201219542240
:1019300079D1B71401D322C250C254C22812191649
:10194000AF3E22758C00758A00D28C22F582E43479
:1019500000F583227993777FC20522D24FD251229C
:101960003401F583E022A42DFDE5F03CFC87F02254
:10197000F536F537F538F539220FBF00010E229004
:10198000017CE0B55F01D322247CF58222F7E55A81
:0B19900024FFB409002279C177002277
:00000001FF
